:1000000001308A0004290000173084000008031919
:10001000172801308D008C018C0B0C288D0B0B28C0
:100020004A308C008C0B12281528800B09280800F8
:100030008316861083128614831606118312061502
:1000400083160612831206168316061383120617EA
:1000500083168612831286168316861383128617DA
:1000600004309600E13097000420960B3228831666
:1000700086108312861083160611831206118316CA
:1000800006128312061283160613831206138316B2
:1000900086128312861283168613831286130F2903
:1000A000831686108312861083160611831206119A
:1000B0008316061283120612831606138312061382
:1000C0008316861283128612831686138312861372
:1000D0002929170807398C00170C8D008D0C8D0C01
:1000E0001F308D050D081807840000088D008C0A4C
:1000F0007A288D0C8C0B792808001E0807398C0093
:100100001E0C8D008D0C8D0C1F308D050D082007E9
:1001100084008D018D0A8C0A8E288D0D8C0B8D2804
:100120009F08031996280D08800499288D090D0849
:10013000800508001D0BA8281C089E0001309F00A8
:10014000A0017D201C089E009F018030A0007D2022
:100150009D08031DB6281C089E009F01A0017D205C
:100160001C089E009F018030A0007D2008003130D7
:100170009C0018089D009A2032309C0019089D00B0
:100180009A201A10180BC728190BC7281A14003008
:100190001A1801309B0036309C001B089D009A20E5
:1001A00000301A1801308D00402934309C001708A7
:1001B0009D009A201810170BDE28181097080319B5
:1001C0001814003018180130990035309C001908B7
:1001D0009D009A200030181801308D004E291A1009
:1001E000180BF3281A14190BF6281A1400301A18D1
:1001F00001309B0037309C001B089D009A20003086
:100200001A1801308D005E2903081F39830004305D
:100210009600E13097000420960B09291828043035
:100220009600E13097000420960B1129553091007B
:10023000333092000F30930094011408073C031CE4
:10024000672904309600FA3097000420960B232982
:1002500050281408970011309800692000300D18BC
:100260000130960014089700123098006920003081
:100270000D18013097001608980017089900B72844
:1002800015100D18151414089700133098006920E4
:1002900000300D18013096009700D52895100D18E4
:1002A0009514003015180130960000309518013073
:1002B00097001608980017089900EF280430960058
:1002C000FA3097000420960B6029940A1D291C29F6
:0202D0006300C9
:02400E00F13F80
:00000001FF
